:100000000C9447000C946F000C946F000C946F00DC
:100010000C946F000C946F000C946F000C946F00A4
:100020000C946F000C946F000C946F000C946F0094
:100030000C94F9160C946F000C946F000C944717F5
:100040000C946F000C946F000C946F000C946F0074
:100050000C946F000C946F000C946F000C946F0064
:100060000C946F000C946F000C946F000C946F0054
:100070000C946F000C946F000C946F000C946F0044
:100080000C946F000C946F000C946F00781711247F
:100090001FBECFEFD0E1DEBFCDBF19E0A0E0B1E0E1
:1000A000EEECF2E300E00BBF02C007900D92AC3A19
:1000B000B107D9F71AE0ACEAB9E001C01D92A53545
:1000C000B107E1F710E0CEE8D0E004C02297FE01CE
:1000D0000E946319CC38D107C9F70C946D170C94A2
:1000E000000011BA1B9886B3992796958795969527
:1000F0008795817090708823B1F790B31B9A8FEF2A
:1001000081BB892F9927089520E086B3992796957A
:1001100087959695879580959095817090708823A6
:1001200039F021BB1B981B9820B31B9A8FEF81BB22
:10013000822F99270895FB0180818823B1F0DB018C
:100140002C9186B399279695879596958795969540
:100150008795817090708823A1F722BB1A9A1A980C
:100160003196DF018081882359F70895CF92DF927D
:10017000EF92FF920F931F93CF93DF93CDB7DEB72C
:1001800026970FB6F894DEBF0FBECDBFFB01D42E6D
:10019000C22E40E085E08D1508F4D82E7E0108942B
:1001A000E11CF11C870134E0CF016AE070E00E949D
:1001B0002B19282FCF016AE070E00E942B19FB0158
:1001C000205DD8012D938D01315037FFEDCF3D2DAE
:1001D000315090E0442341F4CC2031F4F701E30F97
:1001E000F11D80818033C1F091E0492F9923B9F04E
:1001F000F701E30FF11DE08186B399279695879566
:100200009695879596958795817090708823A1F72C
:10021000E2BB1A9A1A9803C0332339F7E5CF332388
:10022000B9F626960FB6F894DEBF0FBECDBFDF91AC
:10023000CF911F910F91FF90EF90DF90CF90089595
:100240005F926F927F928F929F92AF92BF92CF9266
:10025000DF92EF92FF920F931F93CF93DF93CDB76F
:10026000DEB72B970FB6F894DEBF0FBECDBF6A0185
:100270007B01822E502E99248AE0821708F4882E62
:100280003E010894611C711C530109E0C701B601CD
:100290002AE030E040E050E00E943F19DC01CB0151
:1002A000182FC701B6012AE030E040E050E00E947C
:1002B0003F1969017A01105DF50111935F01015049
:1002C00007FFE4CF082D015090E0992041F455201C
:1002D00031F4F301E00FF11D8081803309F091E0EA
:1002E000992E992399F0F301E00FF11DE08186B377
:1002F0009927969587959695879596958795817078
:1003000090708823A1F7E2BB1A9A1A980023D9F6B5
:100310002B960FB6F894DEBF0FBECDBFDF91CF9105
:100320001F910F91FF90EF90DF90CF90BF90AF9013
:100330009F908F907F906F905F9008958F929F9283
:10034000AF92BF92DF92EF92FF920F931F93CF93E2
:10035000DF93CDB7DEB75C01062F8DB69EB6663053
:1003600008F005E06DB77EB7601B71090FB6F89411
:100370007EBF0FBE6DBFEDB6FEB60894E11CF11C4A
:1003800010E0D12E1017A0F121E030E040E050E065
:10039000DD2021F01230A0F1115001C0102F1150BA
:1003A000F701E10FF11D808180539927829FB001F1
:1003B000839F700D929F700D1124460F571FC90126
:1003C000880F991F880F991F880F991F820F931FFD
:1003D000280F391F112319F713C08D3071F0F70161
:1003E000E10FF11D80831F5F101770F6DD2061F6AD
:1003F000C5010E9471008A3081F7E1E0DE2EF3CF63
:100400000FB6F8949EBE0FBE8DBECA010FB6F8940B
:100410009EBE0FBE8DBEDF91CF911F910F91FF90B9
:10042000EF90DF90BF90AF909F908F9008952F92A4
:100430003F925F926F927F928F929F92AF92BF9204
:10044000CF92DF92EF92FF920F931F93CF93DF93A0
:10045000CDB7DEB78C01862E2DB63EB68AE0861764
:1004600008F4882E8DB79EB7881991090FB6F894B5
:100470009EBF0FBE8DBF6DB67EB60894611C711C09
:100480009924592C981408F447C0A1E0EA2EF12CC5
:10049000012D112DAA24BB246501552031F091E0D6
:1004A000991508F041C09A9401C0982C9A94F301D0
:1004B000E90DF11D808180539927AA27BB27BC0134
:1004C000CD01A80197010E940C19DC01CB01A80EF7
:1004D000B91ECA1EDB1ED801C701F3E0880F991FA1
:1004E000AA1FBB1FFA95D1F78E0D9F1DA01FB11F2C
:1004F000E80EF91E0A1F1B1F9920C1F615C08D308A
:1005000081F0F301E90DF11D80839394981408F0B4
:10051000BCCF552009F0B9CFC8010E9471008A30C4
:1005200071F7B1E05B2EF1CF0FB6F8943EBE0FBE6F
:100530002DBEC601B5010FB6F8943EBE0FBE2DBE4E
:10054000DF91CF911F910F91FF90EF90DF90CF90AF
:10055000BF90AF909F908F907F906F905F903F90F3
:100560002F90089580E090E0089580E090E0089555
:10057000089508950895089508955F926F927F9267
:100580008F929F92AF92BF92CF92DF92EF92FF92A3
:100590000F931F93CF93DF93EC017A018B01522EBF
:1005A00094E0EE0CFF1C001F111F9A95D1F7370144
:1005B000480181E0A82EB12CE881F9810190F081F9
:1005C000E02D6A2DCE0109956C01E881F981028048
:1005D000F381E02DCE010995AA27BB278E159F0533
:1005E000A007B10730F50894A11CB11CE881F9817E
:1005F0000190F081E02D6A2DCE0109956C010097E4
:1006000009F452C09C0144275527C401B3010E943C
:100610003F1979018A01E881F9810280F381E02D97
:10062000CE010995AA27BB278E159F05A007B10704
:10063000D0F282E0E816F1040105110528F00894D3
:10064000E108F10801091109C601AA27BB27A80181
:1006500097012F5F3F4F4F4F5F4FBC01CD010E946D
:100660000C193B014C0114E096948794779467949D
:100670001A95D1F7E881F9810480F581E02D6A2D82
:10068000CE010995E881F9810680F781E02DCE0140
:100690000995E881F9810084F185E02DB701CE014B
:1006A0000995552089F009C00FEFE02EF12C012D9E
:1006B000112D0894A108B1087FCFE881F981028447
:1006C000F385E02DCE010995E881F9810484F58553
:1006D000E02DCE010995C401B301DF91CF911F91A7
:1006E0000F91FF90EF90DF90CF90BF90AF909F90D1
:1006F0008F907F906F905F90089580E090E06130E0
:1007000069F0623071F0633079F0643099F06530EF
:1007100071F0663091F0673099F0089581E090E0D3
:10072000089588E090E0089580E290E0089580E8E0
:1007300090E0089580E490E0089580E091E00895CD
:1007400080E094E008958FEF90E00895362F23B76E
:10075000287F3770232BFC012383089561BF089500
:10076000FC0183818860838383818F7B83830895E9
:10077000FC01838183BF089587B7826087BF089596
:1007800080E090E0613049F0623051F0633059F020
:10079000643079F0653051F0089581E090E008957B
:1007A00088E090E0089580E490E0089580E094E08F
:1007B000089580E091E008958FEF9FEF0895362F20
:1007C0002EB5287F3770232BFC01268308957BBD2F
:1007D0006ABD0895FC0186818F7E8683868188604C
:1007E000868384818D7F848384818E7F8483089532
:1007F000FC0184818FBD86818EBD089587B780619D
:1008000087BF089580E090E0613049F0623051F098
:10081000633059F0643079F0653051F0089581E02B
:1008200090E0089588E090E0089580E490E00895D5
:1008300080E094E0089580E091E008958FEF9FEFCD
:100840000895362F20918A00287F3770232BFC01D2
:100850002683089570938700609386000895FC01B5
:1008600086818F7E868386818860868384818D7F62
:10087000848384818E7F84830895FC0184818093A6
:100880008B00868180938A00089580917D0080612D
:1008900080937D000895843050F49927880F991F24
:1008A000880F991F880F991F80509F4F089580E0EF
:1008B00091E00895843068F4E82FFF27EE0FFF1FC2
:1008C000EE0FFF1FEE0FFF1FE050FF4F85819927AE
:1008D00008958091050199270895843068F4E82FE0
:1008E000FF27EE0FFF1FEE0FFF1FEE0FFF1FE05061
:1008F000FF4F8681992708958091060199270895D1
:10090000843068F4E82FFF27EE0FFF1FEE0FFF1F64
:10091000EE0FFF1FE050FF4F8781992708958091C8
:100920000701992708950E94F61708950E94EE176F
:1009300099270895FC01DC01A859BF4F1C92108231
:10094000DC01A959BF4F1C92DC01AB59BF4F8F5B33
:100950009F4F8D939C93CF0101962FE0EB5BFF4F50
:10096000819391932150049627FFFACF08950F9316
:10097000DC01EC91E03178F5FF27EE0FFF1FEE0F61
:10098000FF1FEA0FFB1F62838C91E82FFF27EE0FFA
:10099000FF1FEE0FFF1FEA0FFB1F41838C91E82F13
:1009A000FF27EE0FFF1FEE0FFF1FEA0FFB1F238332
:1009B0008C91E82FFF27EE0FFF1FEE0FFF1FEA0FAE
:1009C000FB1F04838C918F5F8C93FD01E959FF4FCE
:1009D0008081800F80830F910895CF93DF93FB0177
:1009E000DA0180E090E03181EA012981321729F0B3
:1009F000231748F08FEF9FEF08C060814C91641778
:100A000021F06417B8F781E090E0DF91CF9108956D
:100A10006F927F928F929F92AF92BF92CF92DF920E
:100A2000EF92FF920F931F93CF93DF937C01FC0112
:100A3000808166247724C82EDD240894C108D1085B
:100A40004601AA24BA2C681479049CF580E090E051
:100A500008C0B3948B2D992787FD90958C159D0523
:100A600044F5880F991F8E0D9F1D8C01095B1F4F48
:100A7000EC01CB5BDF4FF8014081518168817981C6
:100A8000C7010E94ED048F5F9F4F19F728813981BC
:100A9000F80180819181888399832083318321E0CB
:100AA000A22EB3948B2D992787FD90958C159D05CB
:100AB000C4F2AA2031F6DF91CF911F910F91FF90E0
:100AC000EF90DF90CF90BF90AF909F908F907F90EE
:100AD0006F900895CF93DF93DC01EC01CB59DF4F8A
:100AE0008F5B9F4F8883998320E0522F922F3C91F8
:100AF000131630F01FC09F5F9317E0F42223D1F448
:100B0000E92FFF27EE0FFF1FEA0FFB1FEB5BFF4FE5
:100B10000190F081E02D8181861769F7541729F043
:100B20005F5F9F5F931750F305C021E0E883F9836F
:100B30005F5FF7CFDF91CF910895BF92CF92DF92A1
:100B4000EF92FF920F931F93CF93DF93EC0100E09E
:100B50004881442309F44EC065E6C62ED12CC80E48
:100B6000D91E51E4E52EF12CE80EF91E08C00F5FE6
:100B7000202F3327842F992728173907D8F5F70115
:100B8000041758F4E02FFF27EE0FFF1FEC0FFD1F97
:100B9000EB5BFF4F0190F081E02DD601ED93FC93CC
:100BA00081819927813019F7B0800E948004182F25
:100BB00080E090E00E949604282F88E080936200F5
:100BC000812F992782959295907F9827807F9827EB
:100BD000E0912001F0912101EB0DF11DE80FF91FCB
:100BE000208348810F5F202F3327842F99272817D0
:100BF000390728F2DF91CF911F910F91FF90EF906D
:100C0000DF90CF90BF900895BF92CF92DF92EF9286
:100C1000FF920F931F93CF93DF93EC01199800E09D
:100C20004881442309F449C0A5E6CA2ED12CC80E38
:100C3000D91EF1E4EF2EF12CE80EF91EE0EFBE2EE6
:100C400008C00F5F202F3327842F992728173907D3
:100C5000A0F5F701041758F4E02FFF27EE0FFF1F50
:100C6000EC0FFD1FEB5BFF4F0190F081E02DD601F3
:100C7000ED93FC9381819927823019F710810E94AE
:100C8000800498E090936200992782959295907FD6
:100C90009827807F9827E0912001F0912101E10FB2
:100CA000F11DE80FF91FB08248810F5F202F332715
:100CB000842F99272817390760F2199ADF91CF916D
:100CC0001F910F91FF90EF90DF90CF90BF9008950C
:100CD00020E030E0809161008F7B8093610087B1DC
:100CE000887F866087B9262F206E316010926D0054
:100CF00015BE87E08093640083E080936500809157
:100D000065008260809365008091650081608093BA
:100D10006500809165008B7F809365008091640001
:100D2000826080936400809164008160809364009D
:100D3000809164008460809364002BBB9FEF9ABB1A
:100D400080916500846080936500809165008B7F51
:100D50008093650035BB94BB1BBA9ABB93E180912D
:100D600065008E7F80936500915097FFF8CF369A8B
:100D700021E030E086B19927929582958F7089277E
:100D80009F7089278227932780FDF4CF24B135B146
:100D9000349A809165008E7F809365008091650014
:100DA0008160809365008EE080936D0080EC85BF4C
:100DB000C90108950E94680620E030E041E0833CCC
:100DC000940710F021E030E08356924010F022E0CA
:100DD00030E0C9010895CF93C62F0E94DA06E0E003
:100DE0008230910519F0019781F402C0EEEF0DC039
:100DF00088E080936200E0912001F0912101EC0FE6
:100E0000F11DE081EE2309F4EFEF8E2F9927CF91AA
:100E10000895CF92DF92EF92FF920F931F93CF939B
:100E20007C010E949A0410E088E6C82ED12CCE0CDA
:100E3000DF1C15C0E82FFF27EE0FFF1FEE0FFF1F6F
:100E4000EE0FFF1FE050FF4F25818681082F412FB5
:100E50006C2FC7010E94B7041F5F1031C0F4612FCF
:100E6000C7010E94EB06C82F20E08823A9F3843035
:100E700008F3022F412F682FC7010E94B704CE3F0D
:100E800059F781E0F60180831F5F103140F3C701FD
:100E90000E940805C7010E949D05C7010E94040623
:100EA000CF911F910F91FF90EF90DF90CF90089519
:100EB0000F931F93CF93DF93CDB7DEB722970FB673
:100EC000F894DEBF0FBECDBF8C01FC0131968FE0E0
:100ED00090E01082118212821382349601972FEFD4
:100EE0008F3F9207B1F7F801EF5BFF4F108211823D
:100EF00012821382C8010E949A0419821A8205C0C4
:100F000089819A81019689839A8389819A81885EF1
:100F10009D4FB0F3C8010E94090722960FB6F894BE
:100F2000DEBF0FBECDBFDF91CF911F910F9108950E
:100F30000F931F93CF93DF93CDB7DEB722970FB6F2
:100F4000F894DEBF0FBECDBF8C01FC0131968FE05F
:100F500090E01082118212821382349601972FEF53
:100F60008F3F9207B1F7F801EF5BFF4F10821182BC
:100F700012821382C8010E949A0419821A8205C043
:100F800089819A81019689839A8389819A81885E71
:100F90009D4FB0F3C8010E94090722960FB6F8943E
:100FA000DEBF0FBECDBFDF91CF911F910F9108958E
:100FB0008091630099278871907095958795959594
:100FC0008795959587959927089580E1809362008C
:100FD000E0912001F091210160830895FC01262F0A
:100FE0002770208381819927880F991F880F991F67
:100FF000880F991F282B622FCF010E94E5070895C3
:10100000EF92FF920F931F93CF93DF93CDB7DEB78D
:1010100022970FB6F894DEBF0FBECDBF8C01FC0146
:10102000E08012821186F2806F2DC8010E94EE07C7
:1010300019821A8289819A8180569A4E50F4898148
:101040009A81019689839A8389819A8180569A4EE2
:10105000B0F3C8010E94D807882341F1F8016281EA
:10106000633020F5823041F141E050E0F8018185A4
:101070009927242F3327822B932B892B09F051E0BA
:10108000F8015187E62FFF27EE0FFF1FE00FF11F3A
:10109000F482F8018281E82FFF27EE0FFF1FE00F97
:1010A000F11F4383F80182818F5F8283F394F7E01D
:1010B000FF1508F0B9CF02C040E0D7CF6E2DC801B0
:1010C0000E94EE0722960FB6F894DEBF0FBECDBF8A
:1010D000DF91CF911F910F91FF90EF900895DC0168
:1010E000FC01339682E090E02FEF1082218332964C
:1010F00001973FEF8F3F9307C1F780916400877F8F
:1011000080936400809164008F7E8093640080915E
:101110006500877F80936500809165008F7E809356
:1011200065001C92FD01118212821186CD010E9480
:1011300000080895DC01FC01339682E090E02FEF77
:1011400010822183329601973FEF8F3F9307C1F7BB
:1011500080916400877F80936400809164008F7E1B
:101160008093640080916500877F80936500809103
:1011700065008F7E809365001C92FD0111821282B2
:101180001186CD010E9400080895CF93DF93DC0102
:10119000EFEFEC018A81681738F4E62FFF27EE0F96
:1011A000FF1FEA0FFB1FE4816E2FCD010E94EE07A7
:1011B000DF91CF910895FC01862F87708183992755
:1011C000880F991F880F991F880F991F2081282B3E
:1011D000622FCF010E94E5070895DC01FC018281A6
:1011E000681748F4E62FFF27EE0FFF1FEA0FFB1FDB
:1011F0008481992708958FEF90E00895DC01FC0128
:101200008281681748F4E62FFF27EE0FFF1FEA0FD1
:10121000FB1F83819927089580E090E008953F9215
:101220004F925F926F927F928F929F92AF92BF92F6
:10123000CF92DF92EF92FF920F931F93CF93DF93A2
:101240003C0149015A0188E080936200662309F05D
:10125000EBC086B399279695879596958795969531
:101260008795817090708823A1F78FEF82BB1A9ABF
:101270001A9886B39927969587959695879596950A
:101280008795817090708823A1F78FEF82BB1A9A9F
:101290001A9886B3992796958795969587959695EA
:1012A0008795817090708823A1F78FEF82BB1A9A7F
:1012B0001A9886B3992796958795969587959695CA
:1012C0008795817090708823A1F78FEF82BB1A9A5F
:1012D0001A9886B3992796958795969587959695AA
:1012E0008795817090708823A1F78FE182BB1A9A4D
:1012F0001A98282D86B39927969587959695879560
:1013000096958795817090708823A1F722BB1A9AD1
:101310001A98292D86B3992796958795969587953E
:1013200096958795817090708823A1F722BB1A9AB1
:101330001A982A2D86B3992796958795969587951D
:1013400096958795817090708823A1F722BB1A9A91
:101350001A982B2D86B399279695879596958795FC
:1013600096958795817090708823A1F722BB1A9A71
:101370001A98C82FD3014C91841708F046C185E60E
:10138000482E512C460C571C01E4802E912C860CC3
:10139000971CE0902001F0902101F401C41758F44B
:1013A000EC2FFF27EE0FFF1FE60DF71DEB5BFF4F46
:1013B0000190F081E02DD201ED93FC935081838167
:1013C000E2812E2F3327B901680F711DCB0126173B
:1013D00037072CF5D901B701650F711DAC01A29536
:1013E000B295B07FBA27A07FBA27A60FB71F2C915E
:1013F00086B399279695879596958795969587951F
:10140000817090708823A1F722BB1A9A1A98EF5F17
:10141000AE2FBB27A417B50714F3D3014C91CF5FB0
:10142000C41708F4BACFF1C062E871E08FE49AE023
:101430000E949B0001E02AE0B501A4018FE49AE03C
:101440000E94200162E871E08FE49AE00E949B0014
:101450003324D3018C91381608F07DC0E5E64E2E7A
:10146000512C460C571C71E4872E912C860C971C2E
:10147000F401381608F076C0E32DFF27EE0FFF1FAA
:10148000E60DF71DEB5BFF4F0190F081E02DD201DF
:10149000ED93FC9350818281282F332743818181F2
:1014A000813009F46BC0022FC22FDD27A42EBB248C
:1014B000CE018A0D9B1DC817D9070CF040C0E52E40
:1014C000FF24DE0110E2A295B295B07FBA27A07F7B
:1014D000BA27E0912001F0912101EE0DFF1DAE0F22
:1014E000BF1F8C91C82E0F5F802F992782959295F0
:1014F000907F9827807F9827E80FF91F8081D82E4A
:1015000021E045E0B6018FE49AE00E94B60086B380
:101510009927969587959695879596958795817045
:1015200090708823A1F712BB1A9A1A980F5FA02F08
:10153000BB27CE018A0D9B1DA817B90724F262E8CC
:1015400071E08FE49AE00E949B003394F301808164
:10155000381608F48DCF65E871E08FE49AE00E94B8
:101560009B0053C0D2018D929C9250818281282F82
:10157000332743818181813009F095CF022FC22F1B
:10158000DD279E01240F311DC217D307C4F6E52EB7
:10159000FF24CE0110E2E90182959295907F982771
:1015A000807F9827E0912001F0912101EE0DFF1D31
:1015B000E80FF91F8081992721E043E0BC018FE407
:1015C0009AE00E94B60086B39927969587959695DE
:1015D000879596958795817090708823A1F712BBA7
:1015E0001A9A1A980F5F802F99278C179D07A4F2DB
:1015F00062E871E08FE49AE00E949B003394F3016B
:101600008081381608F434CFA6CFDF91CF911F9197
:101610000F91FF90EF90DF90CF90BF90AF909F9091
:101620008F907F906F905F904F903F900895FC0156
:10163000E158FF4F10821182128213820895EF92B7
:10164000FF920F931F938C010E945807C80187597E
:101650009F4F0E946F08F894F801E757FF4F1082E0
:10166000F801E657FF4F1082F801E557FF4F10824F
:10167000F801E457FF4F8FE18083F801E857FF4FEF
:10168000A1E0FA2EF082F801E558FF4F1082118296
:1016900012821382C8010E94170BF801ED57FF4F09
:1016A00086EA9EE0A0E0B0E080839183A283B383CA
:1016B000F801E957FF4FF08220E040E45FE160E08D
:1016C00070E088E49AE00E94BD02F3E7EF2EF12C6F
:1016D000E00EF11E20E040E950ED63E070E081E4AF
:1016E0009AE00E94BD02DC01CB01F7018083918367
:1016F000A283B38309581F4F20E040E157E260E026
:1017000070E08AE39AE00E94BD02DC01CB01F8019F
:1017100080839183A283B3838091450A8F7D8093D8
:10172000450A8091450A80618093450A80913E0A6E
:101730008F7D80933E0A80913E0A806180933E0AAD
:1017400080913E0A80938B008091400A80938A00AA
:101750008091450A8FBD8091470A8EBD87B7826010
:1017600087BF80914B0A83BF78941F910F91FF90A0
:10177000EF900895EF92FF920F931F938C010E94B8
:101780005807C80187599F4F0E946F08F894F801C5
:10179000E757FF4F1082F801E657FF4F1082F8011C
:1017A000E557FF4F1082F801E457FF4F8FE1808328
:1017B000F801E857FF4F81E0F82EF082F801E55874
:1017C000FF4F1082118212821382C8010E94170BF0
:1017D000F801ED57FF4F86EA9EE0A0E0B0E080837D
:1017E0009183A283B383F801E957FF4FF08220E091
:1017F00040E45FE160E070E088E49AE00E94BD02AE
:10180000B3E7EB2EF12CE00EF11E20E040E950EDA5
:1018100063E070E081E49AE00E94BD02DC01CB014C
:10182000F70180839183A283B38309581F4F20E07F
:1018300040E157E260E070E08AE39AE00E94BD0276
:10184000DC01CB01F80180839183A283B383809173
:10185000450A8F7D8093450A8091450A8061809377
:10186000450A80913E0A8F7D80933E0A80913E0A10
:10187000806180933E0A80913E0A80938B00809124
:10188000400A80938A008091450A8FBD8091470A63
:101890008EBD87B7826087BF80914B0A83BF7894E3
:1018A0001F910F91FF90EF900895FC01E857FF4FB3
:1018B0008081882309F408958FE49AE00E949B00B8
:1018C00008956AE871E00E94550C0895CF93DF9364
:1018D000EC016CE971E00E94550C8FE49AE00E94E3
:1018E00084008823D1F38B3259F08D3221F0CE0160
:1018F0000E94610C0FC0FE01E857FF4F10820AC022
:10190000FE01E857FF4F81E0808364EB71E0CE0178
:101910000E94550C62E871E0CE010E94550CDF91E7
:10192000CF910895EF92FF920F931F93CF93DF9380
:10193000EC01F42ECE010E94550C40E062E08FE4F1
:101940009AE00E949E018C016CEB71E0CE010E9436
:10195000550C40E063E08FE49AE00E949E01E82E7F
:1019600082E0F81659F1402F6F2DCE010E946A05D2
:10197000FE01EB59FF4FCE018F5B9F4F0190F0812D
:10198000E02DE817F907E9F010818F2D0E948004FF
:1019900098E090936200992782959295907F98277E
:1019A000807F9827E0912001F0912101E10FF11D46
:1019B000E80FF91FE08266EC71E005C080EFE82ACD
:1019C000D2CF6FEC71E0CE010E94550CDF91CF9128
:1019D0001F910F91FF90EF900895CF93DF93EC014B
:1019E00067EE71E00E94550C8FE49AE00E9484003B
:1019F0008823D1F38B3631F08037B1F0CE010E94CD
:101A0000610C23C062EF71E0CE010E94550C41E0F1
:101A1000642F8FE49AE00E949E01682FCE018759BF
:101A20009F4F0E94C50811C06AEF71E0CE010E946D
:101A3000550C41E0642F8FE49AE00E949E01682FCC
:101A4000CE0187599F4F0E94DB0862E871E0CE010A
:101A50000E94550CDF91CF910895CF93DF93EC0155
:101A600065E072E00E94550C8FE49AE00E948400C9
:101A70008823D1F38F3671F0803734F4843689F0BF
:101A8000CE010E94610C16C08637D1F7CE010E94AC
:101A9000ED0C10C041E066E172E0CE010E94920CB4
:101AA00009C042E06EE272E0CE010E94920CCE01CB
:101AB0000E94170B62E871E0CE010E94550CDF9185
:101AC000CF910895FC01E857FF4F8081882309F0EA
:101AD0004FC086B399279695879596958795969545
:101AE0008795817090708823A1F78FEF82BB1A9A37
:101AF0001A9886B399279695879596958795969582
:101B00008795817090708823A1F78FEF82BB1A9A16
:101B10001A9886B399279695879596958795969561
:101B20008795817090708823A1F78FEF82BB1A9AF6
:101B30001A9886B399279695879596958795969541
:101B40008795817090708823A1F78FEF82BB1A9AD6
:101B50001A9886B399279695879596958795969521
:101B60008795817090708823A1F762BB1A9A1A98A2
:101B70000895FC01E857FF4F8081882381F486B3E4
:101B800099279695879596958795969587958170CF
:101B900090708823A1F762BB1A9A1A980895862F2D
:101BA0009927BC018FE49AE00E94B600089540E0B6
:101BB00063E08FE49AE00E949E01682F80E090E04D
:101BC0000E949304089580E090E00E949604992773
:101BD0000895FC01E857FF4F8081882309F5262FDF
:101BE00086B3992796958795969587959695879527
:101BF000817090708823A1F722BB1A9A1A98672FD8
:101C000086B3992796958795969587959695879506
:101C1000817090708823A1F762BB1A9A1A98089570
:101C20008FE49AE00E94B6000895CF92DF92FF926F
:101C30000F931F93CF93DF93EC0166E472E00E9451
:101C4000550C8FE49AE00E9484008823D1F38336F8
:101C500039F0863709F493C0CE010E94610CD4C0DC
:101C60006FE2CE010E94620D67E572E0CE010E9434
:101C7000550C60E772E0CE010E94550CFF244881AC
:101C8000442309F4C1C08E010B591F4F81E4C82EB3
:101C9000D12CCC0EDD1E4AC00E944B04BC01CE01EB
:101CA0000E94550C61EC72E0CE010E94550CD801E7
:101CB000ED91FC918081992721E042E0BC01CE01A9
:101CC0000E94E90D66EC72E0CE010E94550CD8012D
:101CD000ED91FC918281992721E042E0BC01CE0187
:101CE0000E94E90D66EC72E0CE010E94550CD8010D
:101CF000ED91FC918381992721E042E0BC01CE0166
:101D00000E94E90D66EC72E0CE010E94550C62E87B
:101D100071E0CE010E94550CF3942F2D332748819A
:101D2000842F99272817390708F06EC0F601F4169A
:101D300058F4EF2DFF27EE0FFF1FEC0FFD1FEB5B9D
:101D4000FF4F0190F081E02DD801ED93FC9381814C
:101D5000992721E043E0BC01CE010E94E90D6EEC21
:101D600072E0CE010E94550CD801ED91FC91818169
:101D70009927843008F490CF66EC72E095CF6FE23B
:101D8000CE010E94620D61ED72E0CE010E94550C01
:101D9000FF248E0107591F4FF8018281F81640F584
:101DA0008F2D992721E0422FBC01CE010E94E90D21
:101DB00063EE72E0CE010E94550C6F2DC8010E94A7
:101DC000ED08992721E045E0BC01CE010E94E90D14
:101DD0006F2DC8010E94FE08882381F462E871E03B
:101DE000CE010E94550CF394F8018281F816C0F2DE
:101DF00062E871E0CE010E94550C06C066EE72E00A
:101E0000CE010E94550CEACFDF91CF911F910F9127
:101E1000FF90DF90CF900895CF93DF93EC0165EFB3
:101E200072E00E94550C8FE49AE00E94840088239F
:101E3000D1F3893609F443C08A36BCF4813609F4FB
:101E400058C082368CF58F3309F46DC08434A1F408
:101E500068E073E0CE010E94550C6FE2CE010E9453
:101E6000620DCE010E94E30D18C08337A1F18437C3
:101E70003CF0863709F446C0CE010E94610C56C082
:101E80008E36D1F763E273E0CE010E94550C6FE20B
:101E9000CE010E94620D8881992721E043E0682FDE
:101EA000CE010E94B90D42C0843631F765E373E07C
:101EB000CE010E94550CCE010E94D70D37C060E5BF
:101EC00073E0CE010E94550CCE010E949D05CE010B
:101ED0000E9404062BC06AE573E0CE010E94550CF7
:101EE0006FE2CE010E94620DFE01E959FF4F808131
:101EF000D3CF63E773E0CE010E94550CCE010E9460
:101F0000090714C06FE2CE010E94620D6AE771E01A
:101F10008FE49AE00E949B0065E771E08FE49AE00D
:101F20000E949B0003C0CE010E94150E62E871E082
:101F3000CE010E94550CDF91CF910895BF92CF92B0
:101F4000DF92EF92FF920F931F93CF93DF93EC01F9
:101F500066E973E00E94550C8FE49AE00E948400C9
:101F60008823D1F38C3609F444C08D3654F481367D
:101F700009F492C0833609F4D2C0CE010E94610CEC
:101F800049C1823709F499C08737B9F7FE01E8578C
:101F9000FF4F8081882309F011C1F9E8EF2EF12C61
:101FA000EC0EFD1E8E0106571F4F40E063E08FE4EC
:101FB0009AE00E949E019C0188E080936200F701F4
:101FC0004081F8018081992782959295907F98278A
:101FD000807F9827E0912001F0912101E40FF11D0D
:101FE000E80FF91F208362E871E0CE010E94550CD2
:101FF00011C16FE2CE010E94620DFE01E857FF4F52
:102000008081882309F0C0C0FE01E557FF4F108191
:102010006CE8C62ED12CCC0EDD1EF6018081811716
:1020200008F4F8C059E8E52EF12CEC0EFD1E48E04E
:10203000B42EB0926200F7012081612F7727CB0187
:1020400082959295907F9827807F9827E091200134
:10205000F0912101E20FF11DE80FF91F008121E04D
:1020600045E0CE010E94E90D63EE72E0CE010E94D0
:10207000550C802F992721E045E0BC01CE010E943C
:10208000E90D62E871E0CE010E94550C1F5FF60178
:102090008081811770F6BEC064EA73E0CE010E94B1
:1020A000550C8E0106571F4F40E062E08FE49AE026
:1020B0000E949E01F8018083ADC06FE2CE010E94B4
:1020C000620DFE01E857FF4F8081882389F519E8EA
:1020D000E12EF12CEC0EFD1E8E0106571F4F88E0FD
:1020E00080936200F7012081F80180819927829511
:1020F0009295907F9827807F9827E0912001F0911A
:102100002101E20FF11DE80FF91F0081802F9927AF
:1021100021E045E0BC01CE010E94E90D64CF67EBF0
:1021200073E0CE010E94550C8E0107571F4FBCCFA4
:1021300066EC73E0CE010E94550C09E8E02EF12C0C
:10214000EC0EFD1EF7018081992720E042E0BC01E2
:102150008FE49AE00E94B6006CEC73E0CE010E941E
:10216000550C8E0106571F4FF8018081992720E0FA
:1021700042E0BC018FE49AE00E94B60068ED73E093
:10218000CE010E94550CABCF61EE73E0CE010E94F0
:10219000550C79E8E72EF12CEC0EFD1EF70180813D
:1021A000992720E042E0BC018FE49AE00E94B6004B
:1021B00062E871E0CE010E94550C26CF66EC73E018
:1021C000CE010E94550CA9E8EA2EF12CEC0EFD1E62
:1021D000F7018081992720E042E0BC018FE49AE07A
:1021E0000E94B6006CEC73E0CE010E94550C8E018B
:1021F00006571F4FF8018081992720E042E0BC017B
:102200008FE49AE00E94B60069E074E0CE010E947B
:10221000550CCBCE62E871E0CE010E94550CDF91E7
:10222000CF911F910F91FF90EF90DF90CF90BF90D3
:10223000089564E174E08FE49AE00E949B006BE1F2
:1022400074E08FE49AE00E949B0062E871E08FE402
:102250009AE00E949B0064E174E08FE49AE00E949F
:102260009B0067E274E08FE49AE00E949B0062E8C2
:1022700071E08FE49AE00E949B0064E174E08FE4D7
:102280009AE00E949B0068E374E08FE49AE00E9469
:102290009B0062E871E08FE49AE00E949B0064E199
:1022A00074E08FE49AE00E949B0068E474E08FE49D
:1022B0009AE00E949B0062E871E08FE49AE00E943D
:1022C0009B0064E174E08FE49AE00E949B006DE55E
:1022D00074E08FE49AE00E949B0062E871E08FE472
:1022E0009AE00E949B0064E174E08FE49AE00E940F
:1022F0009B0068E674E08FE49AE00E949B0062E82D
:1023000071E08FE49AE00E949B0064E174E08FE446
:102310009AE00E949B006DE774E08FE49AE00E94CF
:102320009B0062E871E08FE49AE00E949B000895B0
:102330006AE874E00E94550C64E174E08FE49AE06E
:102340000E949B006EE874E08FE49AE00E949B007C
:1023500062E871E08FE49AE00E949B0064E174E01F
:102360008FE49AE00E949B006DEA74E08FE49AE0AB
:102370000E949B0062E871E08FE49AE00E949B005B
:1023800064E174E08FE49AE00E949B006CEC74E0DE
:102390008FE49AE00E949B0062E871E08FE49AE08B
:1023A0000E949B0064E174E08FE49AE00E949B002D
:1023B0006BEE74E08FE49AE00E949B0062E871E0AB
:1023C0008FE49AE00E949B0064E174E08FE49AE05D
:1023D0000E949B0066E075E08FE49AE00E949B00FB
:1023E00062E871E08FE49AE00E949B0064E174E08F
:1023F0008FE49AE00E949B006CE175E08FE49AE024
:102400000E949B0062E871E08FE49AE00E949B00CA
:1024100064E174E08FE49AE00E949B006EE375E053
:102420008FE49AE00E949B0062E871E08FE49AE0FA
:102430000E949B0008956BE575E00E94550C64E1D5
:1024400074E08FE49AE00E949B006FE575E08FE4F2
:102450009AE00E949B0062E871E08FE49AE00E949B
:102460009B0064E174E08FE49AE00E949B006FE7B8
:1024700075E08FE49AE00E949B0062E871E08FE4CF
:102480009AE00E949B0064E174E08FE49AE00E946D
:102490009B0062EA75E08FE49AE00E949B0062E88C
:1024A00071E08FE49AE00E949B0064E174E08FE4A5
:1024B0009AE00E949B0065EC75E08FE49AE00E9430
:1024C0009B0062E871E08FE49AE00E949B0008950F
:1024D00065EE75E00E94550C64E174E08FE49AE0CB
:1024E0000E949B0069EE75E08FE49AE00E949B00D9
:1024F00062E871E08FE49AE00E949B0064E174E07E
:102500008FE49AE00E949B0068EF75E08FE49AE008
:102510000E949B0062E871E08FE49AE00E949B00B9
:1025200064E174E08FE49AE00E949B006FE076E043
:102530008FE49AE00E949B0062E871E08FE49AE0E9
:102540000E949B0064E174E08FE49AE00E949B008B
:1025500067E276E08FE49AE00E949B0062E871E017
:102560008FE49AE00E949B0064E174E08FE49AE0BB
:102570000E949B006FE376E08FE49AE00E949B004C
:1025800062E871E08FE49AE00E949B0064E174E0ED
:102590008FE49AE00E949B0067E576E08FE49AE082
:1025A0000E949B0062E871E08FE49AE00E949B0029
:1025B00064E174E08FE49AE00E949B006BE676E0B1
:1025C0008FE49AE00E949B0062E871E08FE49AE059
:1025D0000E949B0064E174E08FE49AE00E949B00FB
:1025E0006AE876E08FE49AE00E949B0062E871E07E
:1025F0008FE49AE00E949B0008956DE976E00E94C6
:10260000550C64E174E08FE49AE00E949B0061EA5B
:1026100076E08FE49AE00E949B0062E871E08FE42C
:102620009AE00E949B0064E174E08FE49AE00E94CB
:102630009B006EEB76E08FE49AE00E949B0062E8DC
:1026400071E08FE49AE00E949B0008956CED76E0C3
:102650000E94550C64E174E08FE49AE00E949B00B4
:1026600060EE76E08FE49AE00E949B0062E871E001
:102670008FE49AE00E949B0064E174E08FE49AE0AA
:102680000E949B0069EF76E08FE49AE00E949B0035
:1026900062E871E08FE49AE00E949B0064E174E0DC
:1026A0008FE49AE00E949B0064E177E08FE49AE077
:1026B0000E949B0062E871E08FE49AE00E949B0018
:1026C00064E174E08FE49AE00E949B006EE277E0A0
:1026D0008FE49AE00E949B0062E871E08FE49AE048
:1026E0000E949B0064E174E08FE49AE00E949B00EA
:1026F00068E477E08FE49AE00E949B0062E871E072
:102700008FE49AE00E949B0008956AE874E00E94BA
:10271000550C64E174E08FE49AE00E949B0068E647
:1027200077E08FE49AE00E949B0062E871E08FE41A
:102730009AE00E949B0064E174E08FE49AE00E94BA
:102740009B0063E877E08FE49AE00E949B0062E8D8
:1027500071E08FE49AE00E949B0064E174E08FE4F2
:102760009AE00E949B0061EA77E08FE49AE00E9481
:102770009B0062E871E08FE49AE00E949B0064E1B4
:1027800074E08FE49AE00E949B006DEB77E08FE4A9
:102790009AE00E949B0062E871E08FE49AE00E9458
:1027A0009B0064E174E08FE49AE00E949B0062EE7B
:1027B00077E08FE49AE00E949B0062E871E08FE48A
:1027C0009AE00E949B0064E174E08FE49AE00E942A
:1027D0009B0068E078E08FE49AE00E949B0062E84A
:1027E00071E08FE49AE00E949B0008950F931F937D
:1027F000CF938C0160E378E00E94550CC8010E94E1
:1028000019116AE378E0C8010E94550C8FE49AE040
:102810000E948400C82F8823C9F362E478E08FE423
:102820009AE00E949B0062E871E08FE49AE00E94C7
:102830009B00CB3671F1CC36B4F4C43681F0C5368A
:1028400014F5CF33B1F4C8010E949811C8010E9459
:102850001B12C8010E946812C8010E94FD12C80123
:102860000E94261321C0C337C1F0C43734F0C737E4
:10287000C1F0C8010E94610C17C0CD36D1F7C80164
:102880000E94981111C0C636A1F7C8010E94FD121E
:102890000BC0C8010E94681207C0C8010E941B1229
:1028A00003C0C8010E948513CF911F910F91089515
:1028B0000F93FC01E857FF4F8081882309F041C046
:1028C000242F86B399279695879596958795969503
:1028D0008795817090708823A1F722BB1A9A1A9865
:1028E000252F86B3992796958795969587959695E2
:1028F0008795817090708823A1F722BB1A9A1A9845
:10290000262F86B3992796958795969587959695C0
:102910008795817090708823A1F722BB1A9A1A9824
:10292000472F86B39927969587959695879596957F
:102930008795817090708823A1F742BB1A9A1A98E4
:1029400004C08FE49AE00E9420010F9108950F9334
:10295000CF93DF93EC0163E478E00E94550C8FE4A1
:102960009AE00E9484008823D1F3843431F08435C6
:10297000D1F0CE010E94610C34C06BE578E0CE014D
:102980000E94550CFE01E957FF4F0081002309F119
:102990006FE2CE010E94620D21E043E0622FCE0182
:1029A0000E94B90D1EC066E678E0CE010E94550C6B
:1029B0006FE2CE010E94620DFE01ED57FF4F01E074
:1029C00025E04081518162817381CE010E945814BB
:1029D00008C06FE2CE010E94620D21E043E0602F4B
:1029E000DECF62E871E0CE010E94550CDF91CF91FD
:1029F0000F9108950F931F93CF93DF93EC0160E83D
:102A000078E00E94550C8FE49AE00E9484008823AD
:102A1000D1F38436D1F085364CF48F3399F1813679
:102A200009F459C0CE010E94610C69C08237D1F708
:102A3000FE01E558FF4F10821182128213826FE867
:102A400078E0CE010E94550C5AC06AE978E0CE01C8
:102A50000E94550C40E067E08FE49AE00E94170264
:102A6000AB01BC018E0109581F4F20E08AE39AE0B8
:102A70000E94BD02DC01CB01F80180839183A28317
:102A8000B3833DC06FEB78E0CE010E94550C62ED40
:102A900078E0CE010E94550CFE01ED58FF4F00E09A
:102AA0002AE04081518162817381CE010E945814D5
:102AB0006AED78E0CE010E94550CFE01E958FF4F07
:102AC0002AE04081518162817381CE010E945814B5
:102AD00062E871E0B6CF62EE78E0CE010E94550C5C
:102AE00040E067E08FE49AE00E941702AB01BC016E
:102AF0008E010D581F4F20E081E49AE0B9CF62E8C3
:102B000071E0CE010E94550CDF91CF911F910F9182
:102B10000895CF93DF93EC0167E079E00E94550CB4
:102B20008FE49AE00E9484008823D1F3803781F0FB
:102B3000813734F4853659F1CE010E94610C3EC0D4
:102B40008337C1F08437C1F7CE010E94FA1436C032
:102B500087B7806187BF80913E0A80938B00809108
:102B6000400A80938A008091450A8FBD8091470A70
:102B70008EBD24C01EBC10928A0087B78B7F87BF92
:102B800087B78F7E87BF87B7877F87BF17C0FE0154
:102B9000E558FF4F80819181A281B3819C01AD01F5
:102BA0000196A11DB11D80839183A283B383FE0191
:102BB000E857FF4F6081CE010E940F0962E871E083
:102BC000CE010E94550CDF91CF910895CF93DF93F2
:102BD000EC01FC01E957FF4F8081882301F1FE01E0
:102BE000E158FF4F80819181A281B3810196A11D9F
:102BF000B11D80839183A283B383FE01ED57FF4F04
:102C0000208131814281538182179307A407B50740
:102C100030F0CE010E94170BCE010E940406DF9116
:102C2000CF910895EF92FF920F931F93CF9364E19A
:102C300079E00E94550CF1E0EF2EAAE6B1E0FD012B
:102C400001900020E9F73197EA1BFB0BFE2EC0E054
:102C50008D018FE49AE00E947100F80191918F013B
:102C6000292F332727FD3095992787FD9095281721
:102C7000390709F0EE24CF5FCF1558F38E2D992731
:102C8000CF911F910F91FF90EF9008950F931F9395
:102C9000CF93DF93EC016EE179E00E94550C8FE455
:102CA0009AE00E9484008823D1F3843591F0853521
:102CB00044F48F3361F18434E9F1CE010E94610C58
:102CC00049C0843641F18737C1F7CE010E94170B06
:102CD00041C0CE010E9412168823E1F1CE010E946C
:102CE000170B66E379E0CE010E94550C8E010D575B
:102CF0001F4F40E068E08FE49AE00E941702DC0179
:102D0000CB01F80180839183A283B38323C0CE01DA
:102D10000E94A7141FC0CE010E9412168823D1F072
:102D2000FE01E957FF4F10826DE679E0CE010E9467
:102D3000550C10C0CE010E941216882359F0CE0106
:102D40000E94170BFE01E957FF4F81E080836AE87C
:102D500079E0ECCF62E871E0CE010E94550CDF9182
:102D6000CF911F910F910895CF93DF93EC018FE4E2
:102D70009AE00E9484008823D1F38B3641F18C368F
:102D800084F4843661F18536E4F48F3381F4FE01F6
:102D9000E857FF4F8081882349F1CE010E94F61346
:102DA00025C08337C1F0843734F08737E1F0CE0196
:102DB0000E94610C1BC08D36D1F7CE010E9489158F
:102DC00015C08636A1F7CE010E94660C0FC0CE0159
:102DD0000E940C0F0BC0CE010E942D0D07C0CE012A
:102DE0000E949E0F03C0CE010E944616DF91CF9134
:102DF00008951F920F920FB60F9211242F933F93B5
:102E00004F935F936F937F938F939F93AF93BF93F2
:102E1000EF93FF9386B399270024880F991F001C16
:102E2000880F991F001C892F902D81709070882326
:102E3000E9F019988091270A9091280AA091290A0F
:102E4000B0912A0A9C01AD010196A11DB11D80938C
:102E5000270A9093280AA093290AB0932A0A60911E
:102E6000340A8CEA99E00E940F09199AFF91EF91B8
:102E7000BF91AF919F918F917F916F915F914F9192
:102E80003F912F910F900FBE0F901F9018951F929A
:102E90000F920FB60F9211242F933F934F935F938E
:102EA0006F937F938F939F93AF93BF93EF93FF9312
:102EB0008CEA99E00E94E615FF91EF91BF91AF91E6
:102EC0009F918F917F916F915F914F913F912F9142
:102ED0000F900FBE0F901F901895CFEFD0E1DEBF7F
:102EE000CDBF199A19988CEA99E00E94B416F9CFCF
:102EF000BC9ABD9ABE9ABF9A149A159AC49AC59A5A
:102F0000C69AC79A1C9A1D9A1A981B9A129A139AD3
:102F10008FEF81BBBB98BA98119A8EE080936D00B9
:102F200080EC85BF80916100816080936100809119
:102F30006100826080936100809161008460809371
:102F400061008091610088608093610080916100E0
:102F50008061809361001092620080E091E1909323
:102F6000A9098093A8098FEF9FEF9093AB098093F5
:102F7000AA0986E291E09093490A8093480A109248
:102F80004A0A10924B0A10924C0A8AE491E09093FC
:102F9000420A8093410A1092440A1092430A109206
:102FA000450A1092460A1092470A8CE591E09093E8
:102FB0003B0A80933A0A10923D0A10923C0A109202
:102FC0003E0A10923F0A1092400A80E487B987E8CF
:102FD00086B98CEA99E00E94BA0B0895E199FECF78
:102FE0009FBB8EBBE09A99278DB30895E199FECFE0
:102FF0009FBB8EBB6DBB0FB6F894E29AE19A0FBEF1
:103000000895CF93DF939C01029710F422E030E003
:1030100040E050E0E091530AF091540ABF01DA0118
:103020003097B1F0808191818217930709F485C0B0
:103030002817390738F44115510519F084179507F9
:1030400008F4AC01DF010280F381E02D309751F7E5
:1030500041155105B9F0DA01A21BB30B149708F41E
:103060009A01FB01A0E0B0E0672B61F06081718103
:103070006417750709F43FC0DF010280F381E02D7A
:103080003097A1F74091510A5091520A41155105CC
:1030900041F44091A8095091A9095093520A4093D4
:1030A000510AA091AA09B091AB091097D9F0FA0181
:1030B000BD01641B750B6217730788F0D901129666
:1030C0006A177B0760F0420F531F4E5F5F4F5093AC
:1030D000520A4093510A21933193CF0137C080E0C7
:1030E00090E034C0ADB7BEB7E091A609F091A70952
:1030F000AE1BBF0BDCCF2417350769F0421B530B07
:10310000EF01C40FD51F299339934250504040839B
:103110005183CE011BC0109749F022813381129652
:103120002D933C931397CF01029610C04281538197
:103130005093540A4093530AF6CF109771F72281A7
:1031400033813093540A2093530AEDCFDF91CF910E
:103150000895CF93DF93009709F45BC0DC011297C9
:1031600012961D921C9213978091530A9091540AC3
:103170000097D1F1FC0140E050E0EA17FB0710F5A1
:10318000AF010280F381E02D3097B9F7EA01AA83FD
:10319000BB83FA01329628813981E20FF31FEA17C7
:1031A000FB07B9F56D917C911197260F371F2E5FA4
:1031B0003F4F2883398312964D915C9113974A8330
:1031C0005B8327C0ED011296ED93FC9313972D912D
:1031D0003C911197C20FD31FCE0102968E179F0705
:1031E00041F04115510591F6B093540AA093530A4A
:1031F00010C06A817B81260F371F2E5F3F4F2D93B2
:103200003C9311972281338112962D933C9313970F
:10321000E8CFDF91CF910895629FD001739FF001B5
:10322000829FE00DF11D649FE00DF11D929FF00D56
:10323000839FF00D749FF00D659FF00D9927729F8D
:10324000B00DE11DF91F639FB00DE11DF91FBD0118
:10325000CF0111240895AA1BBB1B51E107C0AA1F6F
:10326000BB1FA617B70710F0A61BB70B881F991F27
:103270005A95A9F780959095BC01CD010895A1E2DA
:103280001A2EAA1BBB1BFD010DC0AA1FBB1FEE1FE0
:10329000FF1FA217B307E407F50720F0A21BB30B2B
:1032A000E40BF50B661F771F881F991F1A9469F7A7
:1032B00060957095809590959B01AC01BD01CF0103
:0E32C0000895EE0FFF1F0590F491E02D099484
:1032CE004E4F4E450000000044494F0000010101E1
:1032DE00445653000006041F4144430000061000EC
:1032EE000020000000007D03A303A603B003AE037D
:1032FE00BC03B80300000000B202B502B802B90266
:10330E00BA02BB02BC0200000000C003DC03DF03F4
:10331E00EA03E703FE03F8030000000002041E04A4
:10332E0021042F042A0445043D04506C6561736525
:10333E00446F49740056312E330053435532555362
:10334E0042000A0D000A0D0A0D00556E6B6E6F7766
:10335E006E20436F6D6D616E640A0D0045696E2DB2
:10336E002F41757367616265666F726D61743A0A9B
:10337E000D3F200041534349490A0D000A0D436F8A
:10338E006465203D20000A0D646F6E650A0D000A0B
:10339E000D4361726420646F6573206E6F742065D7
:1033AE00786973740A0D00566964656F3A0A0D3FA9
:1033BE0020004B617274653A200050432D4B616EB4
:1033CE00616C3A200053656E646520446174656ECD
:1033DE003A0A0D3F200044494F20417573676165DD
:1033EE006E6765207365747A656E3A0A0D004456F1
:1033FE0053204175736761656E6765207365747AD6
:10340E00656E3A0A0D000A0D4B617274656E6C6939
:10341E007374653A0A0D004D6573732D20756E64D5
:10342E0020494F2D4B617274656E3A0A0D0A0D00DC
:10343E0054797065204E616D652020204361726461
:10344E0041647220205265674164722020205265CB
:10345E006753697A6520200A0D2D2D2D2D2D2D2DCA
:10346E002D2D2D2D2D2D2D2D2D2D2D2D2D2D2D2D7E
:10347E002D2D2D2D2D2D2D2D2D2D2D2D2D2D0A0DB1
:10348E00002020202000202020202020200020208E
:10349E0000566964656F204B617274656E3A0A0D51
:1034AE000A0D003A200020202120436F6E666C69C1
:1034BE0063742021004B6F6E666967757261746963
:1034CE006F6E3A0A0D3F2000676574204465666191
:1034DE00756C7420666F722044494F2D496E697465
:1034EE003A20004E756D626572206F6620436172E0
:1034FE0064733A20007365742044656661756C745C
:10350E0020666F722044494F2D496E69743A20002F
:10351E00496E697443617264730053697A65206FF2
:10352E0066204461746120526567697374657273B5
:10353E003A20000A0D4175746F6D6174697363688A
:10354E0065204B617274656E65726B656E6E756E1D
:10355E00670A0D0A0D00446961676E6F73653A0A5A
:10356E000D3F200052656769737465722041647265
:10357E006573733A203F0043617264204164726543
:10358E0073733A203F00436172643D002C205265F4
:10359E006769737465723D002C2056616C75653DCC
:1035AE00002D2D2D2D2D2D2D204C6973742052653F
:1035BE006769737465722056616C756573206F66EA
:1035CE002043617264203D20002C2056616C75658D
:1035DE003D203F00202020202020006D094D6573E6
:1035EE0073756E67656E00730953656E6465206151
:1035FE006E204B61727465006B094B6F6E66696766
:10360E0075726174696F6E00660945696E2D2F4182
:10361E00757367616265666F726D617400640944EB
:10362E006961676E6F736500770944565320576161
:10363E00746368646F672054696D6572003F094159
:10364E006C6C20546F70696373006D0A0D007464A6
:10365E00203C542F75733E092D3E204456532D4D5C
:10366E00657373696E74657276616C6C007461203B
:10367E003C542F75733E092D3E204144432D4D651C
:10368E007373696E74657276616C6C00743F202082
:10369E002020202020093C2D204D657373696E7407
:1036AE00657276616C6C652F7573007472202020C4
:1036BE00202020200920202054696D657374616DCF
:1036CE0070203D2030006520202020202020200961
:1036DE003C2D204D65737377657274007020202029
:1036EE002020202020093C2D204D657373776572B4
:1036FE00746520706572696F646973636800732006
:10370E00202020202020200920202073746F70702C
:10371E00204D657373776572746500730A0D0073BF
:10372E0064203C6E723E203C76616C3E092D3E203C
:10373E0052656C616973206175662044565300733F
:10374E006F203C6E723E203C76616C3E092D3E2011
:10375E004175736761656E676520617566204449C2
:10376E004F00766B202020202020202020202009B2
:10377E002D3E20566964656F204B6162696E656EE1
:10378E007761686C00767020202020202020202079
:10379E002020092D3E20566964656F2050432D4B25
:1037AE00616E616C006B0A0D00762020093C2D20A5
:1037BE0056657273696F6E006109092020204B6196
:1037CE007274656E2065726D697474656C6E0064DA
:1037DE002020092D3E2044494F2D44656661756CAD
:1037EE007476616C756500442020093C2D20444997
:1037FE004F2D44656661756C7476616C75650069F4
:10380E0009092020204B617274656E20696E6974FF
:10381E0069696572656E006E2020093C2D204B6132
:10382E007274656E616E7A61686C00732020093C5B
:10383E002D2047726F6573736520526567697374C7
:10384E00657262657265696368003F6320093C2D8D
:10385E00204B617274656E6C6973746500660A0D37
:10386E00002B0945696E2D2F417573676162656680
:10387E006F726D6174203D204153434949002D09FB
:10388E0045696E2D2F41757367616265666F726D46
:10389E006174203D2042696E61657200640A0D00FC
:1038AE0063203C76616C3E092D3E204B617274653F
:1038BE006E616472657373650061203C76616C3E67
:1038CE00092D3E2052656769737465726164726575
:1038DE007373650072202020202020093C2D205279
:1038EE0065676973746572696E68616C74007720C0
:1038FE002020202020092D3E2052656769737465B3
:10390E0072696E68616C74006C2020202020200982
:10391E003C2D20616C6C652052656769737465720D
:10392E00696E68616C746500772020092020202064
:10393E00636C6561722044565320576174636864EA
:10394E006F670064202020202020200964697361A5
:10395E00626C6520445653205761746368646F67C8
:10396E00004420202020202009656E61626C6520B5
:10397E00445653205761746368646F670054202067
:10398E002020202020092D3E2044565320576174BC
:10399E006368646F672054696D6572706572696FD4
:1039AE0064003F5420202020202020093C2D20445C
:1039BE005653205761746368646F672054696D6550
:1039CE0072706572696F64003F44202020202020B1
:1039DE0020093C2D20445653205761746368646F50
:1039EE00672054696D657220656E61626C65640056
:1039FE000A0D48656C700A0D2000546F70696320C3
:103A0E003F0000445653205761746368646F67200B
:103A1E0053746174653A0A0D3F2000656E61626CE5
:103A2E006564203D2000506572696F642028696EC0
:103A3E002038206D7320537465707329203D20004B
:103A4E007365742054696D65723A0A0D3F200054F7
:103A5E00696D65203D20300A0D00445653204D659A
:103A6E007373696E74657276616C6C2F7573202832
:103A7E00302E2E3430303030303029203A20004D68
:103A8E00657373696E74657276616C6C652F757390
:103A9E003A000A0D4144433A20000A0D4456533A67
:103AAE002000414443204D657373696E74657276D0
:103ABE00616C6C2F75732028302E2E3430303030E0
:103ACE00303029203A20004D657373756E673A0ABF
:103ADE000D3F200050617373776F72643A00445645
:103AEE00532D5761746368646F672054696D6572F6
:103AFE003A0A0D3F200044565320576174636864A0
:103B0E006F6774696D657220506572696F642069A4
:103B1E006E2038206D732D53746570732028302EEF
:103B2E002E3430303030303029203A200044565375
:103B3E002D5761746368646F6774696D6572206474
:103B4E00697361626C65640A0D004456532D5761AA
:103B5E00746368646F6774696D657220656E616207
:0C3B6E006C65640A0D002000550A000080
:013B7A00004A
:00000001FF
